:10000000C8280408920026088400F030A3050830B0
:10001000930003100318A30A1B20920C930B0A28C9
:100020000000971A230C1B20C62003141B201B085A
:100030008F001A086E288413971F2A2800082404AA
:10004000171F24068000841700082404031C2406BC
:100050008000352800082404031C2406171B2406EE
:100060008000841724098005352817081F39FF3EB2
:100070008D001608F53E03188D0A00007B28A31397
:1000800015080319A3170530940027308F0010308E
:10009000552003308F00E83055208F016430552003
:1000A0008F010A30552010085C288E0011088D0041
:1000B00010088C00A2200C088C0094030319A313D1
:1000C0001508031966281402031808000C08031DFC
:1000D000A313A31B0800303EBE288F018E00FF3003
:1000E0008E07031C8F07031CC32803308D00DF30ED
:1000F0007B206F288D01E83E8C008D09FC30031CAD
:1001000084288C07031881288C0764008D0F8128B0
:100110000C188A288C1C8E2800008E2808008E005F
:100120000130922894000F080D02031D99280E0833
:100130000C02043003180130031902301405031DAA
:10014000FF30C32810309200910190010D0D900DE9
:10015000910D0E0890020F08031C0F0F9102031857
:10016000B8280E0890070F0803180F0F9107031007
:100170008C0D8D0D920BA6280C08C32884001D0839
:100180008A001C0882008313031383126400080092
:1001900083161030850001308600811383127B297D
:1001A00064000618D0280130A800A90128088C0096
:1001B00029088D008F010D308F20031DE828643041
:1001C0007A2064000618D028A80A0319A90FD62897
:1001D000C8307A206400061CD02864307A2064007D
:1001E000061CD02801308D0090307B20640006185A
:1001F000D02801308D0090307B200030061801306F
:10020000AB0001308D0090307B206400061CD028AC
:1002100001308D0090307B2064000618D02801301A
:100220008D0090307B20003006180130AC0001308A
:100230008D0090307B206400061CD02801308D009A
:1002400090307B2064000618D02801308D0090305B
:100250007B20003006180130AD0001308D00903059
:100260007B206400061CD02801308D0090307B205C
:1002700064000618D02801308D0090307B200030BB
:1002800006180130AE0001308D0090307B206400F4
:10029000061CD0280800AA0164002B08013C031D9D
:1002A00053290130AA0064002C08013C031D5A297F
:1002B0000230AA0764002D08013C031D61290430A7
:1002C000AA0764002E08013C031D68290830AA070C
:1002D00008000530A6000830A400543096009701AD
:1002E0009A019B0195012A089000910101309C0020
:1002F0009D013F2008008501860186108316861027
:10030000053083126D20D020861483168610831248
:100310004B21692101308F00F4306E207D2963006C
:020320008F2923
:02400E00F53F7C
:00000001FF
